:100000006F003048000000003201000034010000A1
:1000100000000000000000000000000000000000E0
:1000200000000000000000000000000000000000D0
:10003000800C000000000000800C000000000000A8
:10004000800C0000800C0000800C0000800C000080
:10005000F6050000800C0000800C0000800C000001
:10006000800C0000800C0000800C0000800C000060
:10007000800C0000800C0000800C0000800C000050
:10008000800C0000800C0000800C0000800C000040
:10009000800C0000800C0000800C000000000000BC
:1000A000511126C022C206C4828282441244A24058
:1000B00031018280634E050263C305042E86AA8542
:1000C0007D5515C285466378B6006356C0000606A6
:1000D0008606E36CB6FE014563E4C500918D558D3F
:1000E00085820582F5FA82808682C93F2E858282CA
:1000F0003305A04063D70500B305B040C1B7B305D1
:10010000B0408682653F3305A0408282868263C705
:100110000500634905005D372E858282B305B04036
:10012000E35B05FE3305A040513F3305B0408282BA
:10013000000001A0B707EFBE37E700E0938707088C
:100140003CC701A07D151317050141839307F003F8
:1001500063EBE700B70700209387C701AA978823BE
:100160001375F50F828001458280EFF27FF3B7E7C8
:1001700000E03707100023A0E7180F100000EF0081
:10018000704413051003EF0070463745000813054F
:1001900005FCB7040020EF00704901449384C401BA
:1001A000B38784008C2393071400A6979C233745BC
:1001B0000008130505FCA207DD8D2295EF00904A8B
:1001C000090493070004E31DF4FCEF005041CD2027
:1001D000B7E700E03707100023A0E710F9B5EFF20A
:1001E0003FECB7460008370400208147938606FCA1
:1001F0001304C401130600043387D7001823B30582
:10020000F40085071377F70F98A1E397C7FE7C30BA
:100210001307F00F6312F7020567814713074715AD
:10022000930600043306F7000C223306F40085071A
:100230000CA2E399D7FE153F0347F403B70700204C
:1002400085461377F70F9387870163E4E60098A349
:10025000A9BD23800700EDBF9307F5FF13970701A2
:1002600041839307F00363E4E704EFF27FE3B7070A
:100270000020A1469387C7016315D5026393A502A9
:10028000856601479386461513060004B385E6008C
:100290008821B385E700050788A1E319C7FEF1357A
:1002A00029B5BA979823E38DE5FE8CA3CDBF828054
:1002B000EFF21FDF23A40184239C0184A382018425
:1002C000238B0184B7070040DE331145C207C18389
:1002D0002396F184EF00702EC9BBEFF27FDC1C2166
:1002E0000D477111AA8493F7F70F6374B70A183199
:1002F0001394870013740430598C9306400713F746
:10030000470F05046312D702A18B99C7EF006078ED
:10031000AC202285913791A022852D35BC20631E0B
:10032000F502EF00007715A893F7C70F13078007B2
:100330006395E7023C21228593F7F70F3EC01935FC
:10034000B8208247418B9D8B19EBB820B357F540FD
:10035000858B0D83058BE386E7FC1101B9B33EC0A5
:10036000EF0020738247B8208544B394F400E20480
:1003700093778700E184228591C7E933458D937592
:10038000F50F41BFC13393C4F4FFE98C93F5F40F2B
:1003900049B7E394E5FC13F7070F93060007E31E44
:1003A000D7FA13F777009546631AD7001C31370741
:1003B000002093F7F70F2300F700A5B793F6470047
:1003C0009DE2B706002003C506000A0575153A959B
:1003D0004205418159D1A18B95C72AC0EF00606BBE
:1003E0008C30024505BF9146630AD70099466309E0
:1003F000D7009D462145E312D7F6F1BF7545E1BF11
:100400001D45D1BF81339C3019BF8280EFF25FC997
:10041000B307C5009C231307F00393F7F70F639707
:10042000E708130726006353B70805062A96182223
:100430001C2285469354770013F4F707631ED400FB
:10044000A38D0184238D018423860186B7070020B4
:10045000A3809700F929B1A009C49307F4FF13F40E
:10046000F70FB706002083C62600639D960283C659
:10047000B1858DEA0DC81305F002E93109CD0546B5
:100480001305F0022386C18675399316250036952B
:1004900006052397A186B7070020A3809700238D28
:1004A000818421B16DF823860186F5B713F7070C17
:1004B00093060004631AD70693D657401397170084
:1004C0009187798B858BD98F1387E7FF1377F70F88
:1004D000854593F41600E3F5E5F6014463F7F5006E
:1004E0009387D7038A0713F4F70FB707002083C752
:1004F00027006397970283C7B1859DE31DC013054D
:10050000F002893149D905471305F0022386E186B7
:100510001539131725003A9506052397A186A5BF1F
:100520003DF82386018685BF13F7070E9306000862
:10053000631AD70213D74740058B238EE18413D764
:100540003740058BA381E18613D72740058B238194
:10055000E18613D71740058BA380E186858B238026
:10056000F186CDBD13F7070F9306000B6315D70275
:1005700013D73740058BA383E18613D72740058B1C
:100580002383E18613D71740058BA382E186858BF1
:100590002382F186C1B59306000A6315D70213D7EB
:1005A0003740058BA38FE18413D72740058B238F1A
:1005B000E18413D71740058BA38EE184858B2384B8
:1005C000F18649BD13F7C70F9306C00EE31BD7ECA6
:1005D00013073600E357B7EC130716002A971823C2
:1005E00009062A96139587000C2213750530598D3C
:1005F00005059D317DB57111114522C0EF00007ACE
:10060000630D050C1145EF00407BB7070040DA335E
:100610009387C18482234207418333048740420485
:100620004180CD4663FB860A37150140914513058D
:1006300005809AA3EF00100E4DE1096713070771BB
:10064000938781846377870023A00700239C01841C
:1006500069A0984385466305D70A25C38946E315F3
:10066000D7FE138661841822133414050607598CAB
:100670001374F40F9386418400A298220507137720
:10068000F70F98A2A146631AD70493865184982243
:10069000954563E1E50298229375F70F13871500DE
:1006A0001377F70F98A214221387018593F6F60F9C
:1006B0002E9714A3054798C30DA093060005138732
:1006C000818563E086021E239306900F63E7F600A0
:1006D0001E238507C207C1831EA3024411017300B4
:1006E000203016232546637AD600894694C3238298
:1006F000018423830184A382018423100700F1BFB6
:100700009306000563F98600094798C32382018494
:1007100023830184D9B7238BE18423A00700239C82
:10072000E18465BFEFF2DF97130141FC0545EF005F
:10073000D001CD216D347D2A854513055002EF008F
:1007400070088565314613848513081093858513D9
:10075000EF007011371501400C1013050580EF00F4
:10076000A07389450145EF00207C41469305C400F4
:100770006810EF00500F68106D2B930740117C86B6
:10078000680085473EC823070100EF00607C85456F
:100790000545EF001005B707002003A54701B74541
:1007A0000F0093850524EFF07F917D15C167FD173C
:1007B000E8824C08370500403ECC231B0100230E85
:1007C0000100EF00F003854537050040EF003008D9
:1007D000B7070040C23342044180B7070040DE3310
:1007E0001307703E818FC207C1836377F70013043C
:1007F000843E42044180ED2C83C7618593F7F70F57
:10080000E9DFB7E700E03707100023A0E7180F1073
:10081000000083C55184814793F4F50F93860185C9
:1008200013F6F70F63669604238B0184A382018479
:10083000B7E700E03707100023A0E71081468147A3
:100840001387F4FF63CEE7027C183E97834787FC4B
:10085000E395D7F88947E3F297F81C82130700075E
:1008600093F6070F6397E602A6854800BD34B5B737
:100870003386D700082250003E9608A285074DB760
:1008800070183E96034686FC850793F7F70FB18EE6
:1008900055BF93F7070C130700086395E70048005E
:1008A000AD3625BF7545EFF0FF891375050215C5F7
:1008B0008D47E384F4F21C8245453EC0EFF09F88EB
:1008C0008247E39CA7F09C8249453EC0EFF09F879A
:1008D0008247E394A7F0094611A81C8205453EC053
:1008E000EFF05F8682470546E399A7EEA6854800AC
:1008F000313EE5B5EFF2CFFA5111854513055003AE
:10090000EF00406CC1473EC485473EC28A85D94747
:10091000371501407C8023110100BD2B37150140A4
:1009200089478A85130505807C80BD2331016FF0DE
:10093000CFF7EFF2EFF6B7070020754583C4270025
:10094000EFF05F80058919C193C4140003C4C18509
:1009500011C81305100299E013052002EFF08FFE75
:100960001374F50F83C7018681CB13053002EFF0B6
:100970006FFD498C1374F40F83C7118681CB130567
:100980004002EFF02FFC498C1374F40F83C72186CB
:1009900081CB13055002EFF0EFFA498C1374F40F7A
:1009A00083C7318681CB13056002EFF0AFF9498C24
:1009B0001374F40F83C7418681CB13057002EFF0E7
:1009C0006FF8498C1374F40F83C7518681CB1305DC
:1009D0008002EFF02FF7498C1374F40F83C7618600
:1009E00081CB13059002EFF0EFF5498C1374F40FEF
:1009F00083C7718681CB1305A002EFF0AFF4498C59
:100A00001374F40F83C7818681CB1305B002EFF016
:100A10006FF3498C1374F40F83C7D18581CB130511
:100A2000C002EFF02FF2498C1374F40F83C7E185F5
:100A300081CB1305D002EFF0EFF0498C1374F40F63
:100A400083C7F18581CB1305E002EFF0AFEF498C4E
:100A50001374F40F13761400894537150140C12132
:100A600013561440058A9145371501404D291356F8
:100A7000244037150140058A894513050580452125
:100A800013563440058AC1453715014049296FF096
:100A9000CFE1EFF2EFE0B7070040D6330567370448
:100AA0000040C206C182130777385E30958FC207B7
:100AB000C183E37CF7FE0546D94537150140852102
:100AC00037150140054689451305058089295630AB
:100AD000096737060040C206C1821307F7705E320D
:100AE000958FC207C183E37CF7FEA1356FF0EFDB82
:100AF0009387A1869A2319C37D179AA3B70700206D
:100B000003C6170083C6A185B707002083C5270049
:100B1000138727009387B1856395C5008C2363896C
:100B2000D500EFF2EFD710A394A321356FF0EFD7E4
:100B30008280EFF2EFD6371402401C403707FFF8EF
:100B4000414593E717001CC05C40F98F5CC01C4016
:100B50003707F7FE7D17F98F1CC01C403707FCFFD5
:100B60007D17F98F1CC05C4041777D17F98F5CC001
:100B7000B7079F001CC435291C4C93E707021CCC07
:100B8000B717014003A70740938607401377F7F094
:100B900023A0E74003A707401367070823A0E74007
:100BA00089479CCAB7F7FF1F03C5477D9307F00F1E
:100BB0006304F5007D89F52EB72702409843C1767E
:100BC000FD16719B98C398431367170098C3B71716
:100BD0000240D843D8C3D843758FD8C3D843B7068B
:100BE0000001D8C39843558F98C398439316670064
:100BF000E3DD06FED843B7160240719BD8C3D84345
:100C000013672700D8C32147DC42B18BE39EE7FE80
:100C10006FF0AFC9EFF2CFC8371702405C4337041B
:100C200000209146B18B130444016385D700A1468F
:100C30006382D704B7376E01938707601CC0B7166D
:100C40000240DC420840918313F7F700B707002009
:100C500093874700BA978C23DC4293F5F50F93F7FF
:100C600007083357B50081E7EFF04FC52A8718C052
:100C70006FF0AFC35C43B777DC02938707C07DBFDB
:100C800001A097010020938161B9138181FE1305B2
:100C9000000A97F5FF1F9385E53617F6FF1F130629
:100CA000663663FAC5008322050023A055001105AE
:100CB0009105E3EAC5FE170500001305E54D97F51C
:100CC000FF1F9385253417F6FF1F1306263563FA99
:100CD000C5008322050023A0550011059105E3EA14
:100CE000C5FE17F5FF1F13056533938541876377AD
:100CF000B500232005001105E36DB5FEB722000005
:100D000093820288739002308D427390428097F2F2
:100D1000FFFF9382222F93E2320073905230EFF064
:100D20005FE197020000938222A073901234730057
:100D300020305841032305004C45370601409307F6
:100D400006403E979346F3FFB1C583250640F58DD7
:100D50002320B640D043F18ED4C31443B3E66600DB
:100D600014C3184190479346F7FF758E90C7D0473C
:100D7000F18ED4C7144541466399C6009447D98E75
:100D800094C7D447558FD8C78280B6979443558F60
:100D900098C382801C43F58F1CC38280B707014033
:100DA0001387074083A70740584B698F09C77D8D7C
:100DB0003335A000828001458280B707014023AA15
:100DC000A7408280B70767453727024093873712CD
:100DD0005CC3B797EFCD9387B79A5CC38280372700
:100DE00002401C4B93E707081CCB8280B7270240C8
:100DF000C8C78280372702405C470545858B91E74D
:100E000048474189133515000D058280EFF24FA93F
:100E10002A84CD3785476318F50019E0154529A0C8
:100E2000D13F7D14C5BF7DD86FF02FA8EFF24FA73B
:100E3000AA8437050B00D93F91476313F502372485
:100E400002401C4837050B0093E727001CC844C824
:100E50001C4893E707041CC8553F1C48F59B1CC859
:100E60006FF0AFA4EFF2CFA37111AA8409652EC071
:100E7000713F91478245631EF500372402401C48AC
:100E8000096593E717001CC88EA049371C48F99BD9
:100E90001CC811016FF06FA1944593F7060193F2FE
:100EA000F60081C7DC41B3E2F20083D3050093F77B
:100EB000F30FA5C303230500611122C226C0814799
:100EC000130480029304800405473316F70033F7B8
:100ED000C3006312E602939527003D473317B7001E
:100EE0001347F7FF33736700B395B20033E3650030
:100EF000639D860050C985072147E397E7FC1244AC
:100F000023206500824421018280E39696FE10C969
:100F1000DDB7828008456D8D3335A000828019C20F
:100F20000CC982804CC9828037070140144786056E
:100F30008D47B397B70093C7F7FFF58F1CC71C47C2
:100F4000B315B500DD8D0CC7828023A8A1868280F1
:100F500083A60187854718216390F6021C31639CA4
:100F6000D7023C219A0793E707F8B7E600E093F72A
:100F7000F70FBA962380F64085469357570033976C
:100F8000E600544189CE938707048A07B7E600E05C
:100F9000B69798C38280EDF33C219A07F9B79387FF
:100FA0000706B7E600E08A07B69798C30F1000005F
:100FB0008280371702401C430E0593F777F05D8D52
:100FC00008C3828099C5371702401C4F5D8D08CF3A
:100FD0008280B7170240984F1345F5FF798D88CF6F
:100FE000828099C5371702405C4F5D8D48CF828063
:100FF000B7170240D84F1345F5FF798DC8CF8280CF
:101000001E2137370140130707C0C207C18363069B
:10101000E500370700406316E500BA2193F7F7F8BB
:10102000D98FFA2193F7F7CFC207C183D98F1EA1B9
:10103000DE215EB59E211EB5B7370140938707C0FC
:101040006314F5009C251EB985475EA982801E2188
:1010500089C593E717001EA18280C207C183F99B4F
:10106000C207C183CDBFB3C7A5008D8B3307C500B1
:1010700081E78D4763E7C702AA87637EE50A94216B
:1010800085078505A38FD7FEE3EBE7FE82809421D9
:1010900085078505A38FD7FEE3EBE7FE0244110128
:1010A000828093763500AA8789CA942185078505B1
:1010B000A38FD7FE93F63700C5BF9376C7FF13867D
:1010C00006FE63F5C706711122C0C04903A30500DF
:1010D00083A38500C0CB804D23A0670003A34500F8
:1010E00080CFC04D23A2670083A2C50003A30501E2
:1010F00093854502C0CF03A4C5FF23A4770023A690
:10110000570023A867009387470223AE87FEE3EECC
:10111000C7FAE3F3D7F890419107910523AEC7FED4
:10112000CDBF90419107910523AEC7FEE3EBD7FEFB
:10113000E3E7E7F482808280040000000100000001
:101140000400000004000000000000001000000087
:101150000100000003000000FF000A9C00400000A6
:1011600000000000C080000000000000000000003F
:10117000020000000102040810200000000000002E
:101180000000000000000A030E1400000000000030
:04119000000000005B
:10119400010101000102030405060708010203041A
:0811A40005060708006CDC02DF
:00000001FF
